:020000040000FA
:02000000462890
:08000800A0000308A10083120F
:100010000B190D280C182E280028CD30810022083D
:100020001E029F1403191A28031C1B28A20A23026C
:10003000031C2414A20AA203A4182328A50A031946
:10004000A60A0319A414A4192828AC030319A4159B
:100050000B1121088300A00E200E0900CE308F0066
:10006000A41A3728851C4128241AA41624122419FE
:100070003F280130A702031CA802031C24150C1002
:1000800029282416A90A0319A90337288B139021BC
:100090009F218512AA018230AB00851C4A28AA0B39
:1000A0004D28AB0B4D2883169614831205088B152B
:1000B00063008312AA014130AB00AA0B5D28AB0B91
:1000C0005D28851800288316FF23900083122416CC
:1000D000A412A413A90190219F21B221C021CF21F4
:1000E000BD2124137921A41F1622A41BDC21193061
:1000F000290203182417241B0515A41E7728A9011B
:10010000A412241B0E29A41F88280028DC21002803
:100110007921B101B2010130A300A901A412241375
:10012000A41724155030A7004630A8002411A415A8
:10013000FF30AC00A411A41D9B28A414A501A601A6
:100140002D3084002410A412241A71282419862822
:10015000241CA328A4142508B3002608B400A50174
:10016000A601A410A4156430AC00A4110008B500C9
:10017000840A0008B6003402031DC0283508330283
:10018000031CCD283308AA003408AB003508AA02A6
:100190003608031C360AAB02D7283508AA003608F1
:1001A000AB003308AA023408031C340AAB02031064
:1001B000B60CB50C2B083602031DE0282A083502C0
:1001C0000318E4282D308400031CE728840A000863
:1001D000B500840A000884033504031D06290514AC
:1001E0000515A415FF30AC00A411A41DF5280510B9
:1001F0002410A4145F30A500F030A600A410A41CA5
:10020000FF280511241C9128FF219128A41D0629EF
:100210002410A4189D28241C0929AA280630A3000C
:10022000A901A4122417A41324155830A7000230E2
:10023000A8002411A415FF30AC00A411A41D1E2990
:10024000A414A501A601AD01AE012410241A332A7D
:1002500024198628241C2629A4142D08AF002E0852
:10026000B0002508AD002608AE00A501A601A41027
:10027000A4156430AC00A411A41D3C292410A418BA
:100280004429241C3F292C292F0830040319542900
:100290002D08AA002E08AB002F08AD003008AE00D4
:1002A0002A08AF002B08B0008B1383160030AA0079
:1002B0002D3084002A089B0000089A001C15553038
:1002C0009D00AA309D009C149C1864291A081C14D7
:1002D0001A06031D0028840AAA0A04302A02031DF4
:1002E0005A2983128C138B17A901A41629222922BB
:1002F0007128831600309B001C141A08AD000130D1
:100300009B001C141A08AE0002309B001C141A0833
:10031000AF0003309B001C141A08B00083120800C1
:1003200083128B0190019F010730990083168C0185
:10033000810199019F0183128B018C0108008312B6
:100340008B1185018316960195019514811305166D
:100350008514851585120511051083128516051162
:100360000510080083160C139F151F1683129F1388
:100370001F131F159F151F1408000B178B1708005C
:1003800090019016101683160C1083120C108E011B
:10039000CE308F0083160C148312101408008316BD
:1003A0008116811583128B120B11CD3081008316BB
:1003B000811283128B160800AA012A08AB00E029DB
:1003C000E1290511AB0FDF29AB00AB09E729E829CB
:1003D0000515AB0FE629AA0FDD29AA012A08AB00F3
:1003E000F129F2290515AB0FF029AB00AB09F8296B
:1003F000F9290511AB0FF729AA0FEE2908001430CF
:10040000AA000515A4148E30A500FD30A600A41086
:10041000A41C082A0511A4148E30A500FD30A600E6
:10042000A410A41C112AAA0B012A080020222D08BE
:100430002E04031D20222F083004031D2022080053
:10044000A4147730A500EC30A600A4100515A41C58
:10045000272AA4147730A500EC30A600A4100511BB
:10046000A41C302A08000511A4147730A500EC3034
:10047000A600A410A41C3A2A05140515A415FF30E3
:10048000AC00A411A41D422A05110510292229221D
:020490007128D1
:0207FE00803445
:084000000400040001000100AE
:02400E00843FED
:00000001FF
